:020000040000FA
:040000002DEF00F0F0
:0200080014D012
:08001800D8CF81F0E8CF80F0A1
:10002000E0CF82F082C0E0FF80C0E8FF81C0D8FF4F
:100030001000F5CF1FF0F8CF1CF0F7CF1DF0F6CF72
:100040001EF0F2B483ED04F01FC0F5FF1CC0F8FFF2
:100050001DC0F7FF1EC0F6FF1100060EC16E0F0196
:10006000386B396B3A6B3B6B3C6B270E926EF80E1C
:10007000936E030E946E000E956E96849682968013
:10008000720ED36E00EE00F000EC03F080EC04F092
:10009000F28CF28AF28E010E086E010E096E06ECE9
:1000A00003F006EC03F006EC03F000EC08F08BEC38
:1000B00008F0A7EC08F0898614EC09F0118006EC32
:1000C00003F0080EF66E160EF76E000EF86EF0ECEA
:1000D00008F0206A80B0208080B2208280B4208422
:1000E00081B6208620500F0F216E35EC03F0205092
:1000F0000A08100ED8B022C009F0D8A0096ED8B0F6
:1001000023C008F0D8A0086E81AA899881BA89888E
:1001100081A8899681B88986C1EC09F02350300FF7
:1001200062EC08F02250300F62EC08F0DF0E62EC57
:1001300008F0430E62EC08F0200E62EC08F080AA92
:10014000ACEF00F01A0EF66E160EF76E000EF86E9B
:10015000F0EC08F0B4EF00F0280EF66E160EF76E15
:10016000000EF86EF0EC08F020EC03F020EC03F049
:1001700020EC03F020EC03F069EF00F0898834EC08
:0601800003F0C1EF00F0E6
:100600000400EE6AEAA400EF03F01200FF0E0A6E87
:10061000FF0E0B6E0B2E0AEF03F00A2E08EF03F00D
:1006200012000C6EFF0E0D6EFF0E0E6E0E2E16EFEC
:1006300003F00D2E14EF03F00C2E12EF03F0120056
:10064000020E0A6EFF0E0B6E0B2E24EF03F00A2E25
:1006500022EF03F012000000000000000000000084
:1006600000000000000012001200236A226A0A0E35
:10067000215ED8A03FEF03F0232A37EF03F00A0EE4
:060680002124226E12008D
:10090000C30ED56E1200F29407B094EF04F08B96EC
:10091000000EF86E0B0EF76E09C0F6FF0800F5CF5B
:100920008CFF8B84078012008B94000EF86E0B0EE8
:10093000F76E08C0F6FF0800F5CF8CFF8B86079096
:020940001200A3
:100B00003F065B4F666D7D077F6F777C395E79713D
:040B100000400000A1
:10100000156A1580110E136ECBEC08F08BEC08F00E
:101010009BEC08F0C3EC08F093EC08F0ABEC08F0A4
:1010200012002BEC03F02BEC03F02BEC03F02BEC79
:1010300003F08A802BEC03F02BEC03F02BEC03F095
:101040008A902BEC03F02BEC03F02BEC03F0120056
:101050001980198019801980948E948C948A9488B0
:101060008A948A828A802BEC03F082B8FED719908A
:10107000199019901990949E949C949A94981200A7
:101080001A6E28EC08F08A948A928B9E8B9C8B9A1D
:101090008B981AB88B8E1ABA8B8C1ABC8B8A1ABE94
:1010A0008B8811EC08F08B9E8B9C8B9A8B981AB0D6
:1010B0008B8E1AB28B8C1AB48B8A1AB68B8811EC71
:1010C00008F0120011B049EC09F01A6E132E02D08C
:1010D00072EC09F028EC08F08A928A848B9E8B9C33
:1010E0008B9A8B981AB88B8E1ABA8B8C1ABC8B8AF7
:1010F0001ABE8B8811EC08F08B9E8B9C8B9A8B9878
:101100001AB08B8E1AB28B8C1AB48B8A1AB68B8853
:1011100011EC08F01200156A1580110E136E010E05
:1011200040EC08F01200156A1580110E136E020EC5
:1011300040EC08F012000C0E40EC08F01200080E13
:1011400040EC08F012000E0E40EC08F012000C0EFD
:1011500040EC08F012000F0E40EC08F012000E0EEA
:1011600040EC08F01200140E40EC08F01200100ED3
:1011700040EC08F012001C0E40EC08F01200180EB3
:1011800040EC08F01200060E40EC08F01200040ECD
:1011900040EC08F012008A928A9420EC03F006ECEE
:1011A00003F08B8E8B8C8B9A8B9811EC08F020ECD3
:1011B00003F006EC03F08B8E8B8C8B9A8B9811ECE2
:1011C00008F020EC03F006EC03F08B8E8B8C8B9AEE
:1011D0008B9811EC08F020EC03F006EC03F0120001
:1011E000090011A004D0F52AD8B407D0F506F550AF
:1011F000D8B4120062EC08F0F3D7186E0900F50EAF
:10120000F518D8A406D01190F55062EC08F01180C2
:10121000E7D718500A000A00EAD70900F550D8B4F9
:10122000120062EC08F0F9D7000EF86E180EF76E97
:10123000000EF66E400E126E400E40EC08F00900F3
:10124000F5CF1AF028EC08F08A928A848B9E8B9C4A
:101250008B9A8B981AB88B8E1ABA8B8C1ABC8B8A85
:101260001ABE8B8811EC08F08B9E8B9C8B9A8B9806
:101270001AB08B8E1AB28B8C1AB48B8A1AB68B88E2
:1012800011EC08F0122E1FEF09F0800E40EC08F070
:101290001200146E010E176EE10E1418D8B420D08F
:1012A000172AE90E1418D8B41BD0172AF50E1418F3
:1012B000D8B416D0172AFA0E1418D8B411D0172A99
:1012C000FB0E1418D8B40CD0172AF30E1418D8B487
:1012D00007D0172AED0E1418D8B402D014501200FB
:1012E000175012001AC016F015B007D015B211D061
:1012F00015B41BD015B625D01200156A15828A9236
:101300008A94C00E40EC08F0100E136E16C01AF04E
:101310001200156A15848A928A94900E40EC08F0A7
:10132000100E136E16C01AF01200156A15868A92F6
:101330008A94D00E40EC08F0100E136E16C01AF00E
:101340001200156A15808A928A94800E40EC08F08B
:10135000100E136E16C01AF01200B3EC08F0132E24
:10136000ADEF09F0100E136E16C01AF01200156AD8
:1013700015808A928A94800E40EC08F0110E136E4C
:101380001200156A15828A928A94C00E40EC08F009
:10139000110E136E1200156A15848A928A94900EAB
:1013A00040EC08F0110E136E1200156A15868A9231
:0E13B0008A94D00E40EC08F0110E136E12005D
:101600005445535A5400000C537A6F6261746572EA
:101610006D6F737A74E17400000C6E79E172692069
:10162000FFF57A656D00000C74E96C6920FFF57AAE
:06163000656D2000000CB6
:0C1700008182A0A1A2A39A940000000C1A
:10180000000000000000000002040E010F110F0094
:1018100002040E111F100E00050A000E11110E0019
:101820000204111111130D00050A111111130D00FD
:1018300002040E1111110E0002040C0404040E0027
:10184000000FD8A42EEF0CF0000EF86E190EF76EF4
:10185000000EF66E400E126E38EF0CF0000EF86EB1
:10186000190EF76E400EF66E100E126E38EF0CF079
:10187000400E40EC08F00900F5CF1AF028EC08F013
:101880008A928A848B9E8B9C8B9A8B981AB88B8EAB
:101890001ABA8B8C1ABC8B8A1ABE8B8811EC08F092
:1018A0008B9E8B9C8B9A8B981AB08B8E1AB28B8CDA
:1018B0001AB48B8A1AB68B8811EC08F0122E3BEF03
:0A18C0000CF0800E40EC08F012005E
:10190000110E0C0A060E111F1B131B1B1B1B111F94
:10191000110E1E1D1B17001F001D1B1D1E0E111F6B
:101920001D19150D001D1D1F000F011E1E0E111F7C
:1019300019170F010E0E111F02040E010F110F00D7
:10194000110E0E110E0E111F110E0E101E1D131F63
:020000040030CA
:0300010028183C80
:02000500BD81BB
:060008000FC00FE00F40E5
:00000001FF
